Archive member included because of file (symbol)

/opt/gcc-arm-none-eabi-4_7-2013q1/bin/../lib/gcc/arm-none-eabi/4.7.3/armv6-m/libgcc.a(_udivsi3.o)
                              out/cvkbdarm.o (__aeabi_uidiv)
/opt/gcc-arm-none-eabi-4_7-2013q1/bin/../lib/gcc/arm-none-eabi/4.7.3/armv6-m/libgcc.a(_dvmd_tls.o)
                              /opt/gcc-arm-none-eabi-4_7-2013q1/bin/../lib/gcc/arm-none-eabi/4.7.3/armv6-m/libgcc.a(_udivsi3.o) (__aeabi_idiv0)

Discarded input sections

 .data          0x00000000        0x0 out/startup.o
 .bss           0x00000000        0x0 out/startup.o
 .group         0x00000000        0x8 out/vectors.o
 .text          0x00000000        0x0 out/vectors.o
 .data          0x00000000        0x0 out/vectors.o
 .bss           0x00000000        0x0 out/vectors.o
 .group         0x00000000        0x8 out/cvkbdarm.o
 .group         0x00000000        0x8 out/cvkbdarm.o
 .group         0x00000000        0x8 out/cvkbdarm.o
 .group         0x00000000        0x8 out/cvkbdarm.o
 .group         0x00000000        0x8 out/cvkbdarm.o
 .group         0x00000000        0x8 out/cvkbdarm.o
 .group         0x00000000        0x8 out/cvkbdarm.o
 .group         0x00000000        0x8 out/cvkbdarm.o
 .group         0x00000000        0x8 out/cvkbdarm.o
 .group         0x00000000        0x8 out/cvkbdarm.o
 .group         0x00000000        0x8 out/cvkbdarm.o
 .group         0x00000000        0x8 out/cvkbdarm.o
 .text          0x00000000        0x0 out/cvkbdarm.o
 .data          0x00000000        0x0 out/cvkbdarm.o
 .bss           0x00000000        0x0 out/cvkbdarm.o
 .debug_macro   0x00000000      0x7d2 out/cvkbdarm.o
 .data          0x00000000        0x0 /opt/gcc-arm-none-eabi-4_7-2013q1/bin/../lib/gcc/arm-none-eabi/4.7.3/armv6-m/libgcc.a(_udivsi3.o)
 .bss           0x00000000        0x0 /opt/gcc-arm-none-eabi-4_7-2013q1/bin/../lib/gcc/arm-none-eabi/4.7.3/armv6-m/libgcc.a(_udivsi3.o)
 .data          0x00000000        0x0 /opt/gcc-arm-none-eabi-4_7-2013q1/bin/../lib/gcc/arm-none-eabi/4.7.3/armv6-m/libgcc.a(_dvmd_tls.o)
 .bss           0x00000000        0x0 /opt/gcc-arm-none-eabi-4_7-2013q1/bin/../lib/gcc/arm-none-eabi/4.7.3/armv6-m/libgcc.a(_dvmd_tls.o)

Memory Configuration

Name             Origin             Length             Attributes
rom              0x00000000         0x00008000         xr
ram              0x10000000         0x00001000         xrw
*default*        0x00000000         0xffffffff

Linker script and memory map

LOAD out/startup.o
LOAD out/vectors.o
LOAD out/cvkbdarm.o
LOAD /opt/gcc-arm-none-eabi-4_7-2013q1/bin/../lib/gcc/arm-none-eabi/4.7.3/../../../../arm-none-eabi/lib/armv6-m/libstdc++.a
LOAD /opt/gcc-arm-none-eabi-4_7-2013q1/bin/../lib/gcc/arm-none-eabi/4.7.3/../../../../arm-none-eabi/lib/armv6-m/libm.a
START GROUP
LOAD /opt/gcc-arm-none-eabi-4_7-2013q1/bin/../lib/gcc/arm-none-eabi/4.7.3/armv6-m/libgcc.a
LOAD /opt/gcc-arm-none-eabi-4_7-2013q1/bin/../lib/gcc/arm-none-eabi/4.7.3/../../../../arm-none-eabi/lib/armv6-m/libg.a
LOAD /opt/gcc-arm-none-eabi-4_7-2013q1/bin/../lib/gcc/arm-none-eabi/4.7.3/../../../../arm-none-eabi/lib/armv6-m/libc.a
END GROUP
                0x00000000                __main_stack_size = 0x0
                0x00000400                __process_stack_size = 0x400
                [0x00000000]                PROVIDE (__main_stack_size, __main_stack_size)
                [0x00000400]                PROVIDE (__process_stack_size, __process_stack_size)
                0x00000000                __rom_start = ORIGIN (rom)
                0x00008000                __rom_size = 0x8000
                0x00008000                __rom_end = (__rom_start + __rom_size)
                0x10000000                __ram_start = ORIGIN (ram)
                0x00001000                __ram_size = 0x1000
                0x10001000                __ram_end = (__ram_start + __ram_size)
                [0x00000000]                PROVIDE (__rom_start, __rom_start)
                [0x00008000]                PROVIDE (__rom_size, __rom_size)
                [0x00008000]                PROVIDE (__rom_end, __rom_end)
                [0x10000000]                PROVIDE (__ram_start, __ram_start)
                [0x00001000]                PROVIDE (__ram_size, __ram_size)
                [0x10001000]                PROVIDE (__ram_end, __ram_end)

.text           0x00000000      0xf30
                0x00000000                . = ALIGN (0x4)
                0x00000000                __text_start = .
                [0x00000000]                PROVIDE (__text_start, __text_start)
                0x00000000                . = ALIGN (0x4)
 *(.vectors)
 .vectors       0x00000000       0xc0 out/vectors.o
                0x00000000                vectors
                0x000000c0                . = ALIGN (0x4)
 *(.text .text.* .gnu.linkonce.t.*)
 .text          0x000000c0       0x64 out/startup.o
                0x000000c0                Reset_Handler
                0x000000fc                __default_low_level_init
                0x000000fc                low_level_init_1
                0x000000fc                low_level_init_0
 .text.__Default_Handler
                0x00000124        0x8 out/vectors.o
                0x00000124                WAKEUP_PIO0_11_IRQHandler
                0x00000124                TIMER16_0_IRQHandler
                0x00000124                HardFault_Handler
                0x00000124                WAKEUP_PIO0_3_IRQHandler
                0x00000124                SysTick_Handler
                0x00000124                __Reserved_0x1C_Handler
                0x00000124                PendSV_Handler
                0x00000124                UART_IRQHandler
                0x00000124                TIMER32_0_IRQHandler
                0x00000124                WAKEUP_PIO0_10_IRQHandler
                0x00000124                TIMER32_1_IRQHandler
                0x00000124                WAKEUP_PIO0_8_IRQHandler
                0x00000124                __Reserved_0x20_Handler
                0x00000124                __Reserved_0x10_Handler
                0x00000124                PIOINT1_IRQHandler
                0x00000124                CAN_IRQHandler
                0x00000124                SSP0_IRQHandler
                0x00000124                __Reserved_0x34_Handler
                0x00000124                __Reserved_0x30_Handler
                0x00000124                TIMER16_1_IRQHandler
                0x00000124                WAKEUP_PIO0_7_IRQHandler
                0x00000124                ADC_IRQHandler
                0x00000124                SSP1_IRQHandler
                0x00000124                PIOINT2_IRQHandler
                0x00000124                __Reserved_0x18_Handler
                0x00000124                __Reserved_0x28_Handler
                0x00000124                BOD_IRQHandler
                0x00000124                WAKEUP_PIO0_2_IRQHandler
                0x00000124                __Reserved_0x08_Handler
                0x00000124                I2C_IRQHandler
                0x00000124                WAKEUP_PIO0_9_IRQHandler
                0x00000124                __Reserved_0x24_Handler
                0x00000124                WDT_IRQHandler
                0x00000124                SVC_Handler
                0x00000124                __Reserved_0xAC_Handler
                0x00000124                WAKEUP_PIO0_5_IRQHandler
                0x00000124                __Reserved_0x14_Handler
                0x00000124                __Reserved_0x9C_Handler
                0x00000124                WAKEUP_PIO0_1_IRQHandler
                0x00000124                __Reserved_0x98_Handler
                0x00000124                WAKEUP_PIO0_0_IRQHandler
                0x00000124                WAKEUP_PIO0_6_IRQHandler
                0x00000124                WAKEUP_PIO0_4_IRQHandler
                0x00000124                WAKEUP_PIO1_0_IRQHandler
                0x00000124                PIOINT3_IRQHandler
 .text.NVIC_EnableIRQ
                0x0000012c       0x2c out/cvkbdarm.o
 .text.pll_start
                0x00000158      0x104 out/cvkbdarm.o
 .text.PIOINT0_IRQHandler
                0x0000025c      0x1f0 out/cvkbdarm.o
                0x0000025c                PIOINT0_IRQHandler
 .text.set_layout
                0x0000044c       0x38 out/cvkbdarm.o
 .text.map_uncooked
                0x00000484       0x98 out/cvkbdarm.o
 .text.is_first_32
                0x0000051c       0x3c out/cvkbdarm.o
 .text.apply_cap
                0x00000558       0x34 out/cvkbdarm.o
 .text.apply_sh
                0x0000058c       0xfc out/cvkbdarm.o
 .text.apply_ctl
                0x00000688       0x40 out/cvkbdarm.o
 .text.apply_alt
                0x000006c8       0x40 out/cvkbdarm.o
 .text.apply_num
                0x00000708       0x5c out/cvkbdarm.o
 .text.main     0x00000764      0x520 out/cvkbdarm.o
                0x00000764                main
 .text          0x00000c84       0x9c /opt/gcc-arm-none-eabi-4_7-2013q1/bin/../lib/gcc/arm-none-eabi/4.7.3/armv6-m/libgcc.a(_udivsi3.o)
                0x00000c84                __udivsi3
                0x00000c84                __aeabi_uidiv
                0x00000d0c                __aeabi_uidivmod
 .text          0x00000d20        0x4 /opt/gcc-arm-none-eabi-4_7-2013q1/bin/../lib/gcc/arm-none-eabi/4.7.3/armv6-m/libgcc.a(_dvmd_tls.o)
                0x00000d20                __aeabi_ldiv0
                0x00000d20                __aeabi_idiv0
                0x00000d24                . = ALIGN (0x4)
 *(.glue_7t .glue_7)
 .glue_7        0x00000000        0x0 linker stubs
 .glue_7t       0x00000000        0x0 linker stubs
                0x00000d24                . = ALIGN (0x4)
 *(.rodata .rodata.* .gnu.linkonce.r.*)
 .rodata.scankey_e0
                0x00000d24       0x28 out/cvkbdarm.o
 .rodata.apply_sh
                0x00000d4c       0xc8 out/cvkbdarm.o
 .rodata.apply_num
                0x00000e14       0x34 out/cvkbdarm.o
 .rodata.main   0x00000e48       0xe8 out/cvkbdarm.o
                0x00000f30                . = ALIGN (0x4)
 *(.ARM.extab* .gnu.linkonce.armextab.*)
                0x00000f30                . = ALIGN (0x4)
 *(.gcc_except_table)
                0x00000f30                . = ALIGN (0x4)
 *(.eh_frame_hdr)
                0x00000f30                . = ALIGN (0x4)
 *(.eh_frame)
                0x00000f30                . = ALIGN (0x4)
 *(.init)
                0x00000f30                . = ALIGN (0x4)
                0x00000f30                __preinit_array_start = .
 *(.preinit_array)
                0x00000f30                . = ALIGN (0x4)
                0x00000f30                __preinit_array_end = .
                0x00000f30                __init_array_start = .
 *(SORT(.init_array.*))
                0x00000f30                . = ALIGN (0x4)
 *(.init_array)
                0x00000f30                . = ALIGN (0x4)
                0x00000f30                __init_array_end = .
 *(.fini)
                0x00000f30                . = ALIGN (0x4)
                0x00000f30                __fini_array_start = .
 *(.fini_array)
                0x00000f30                . = ALIGN (0x4)
 *(SORT(.fini_array.*))
                0x00000f30                . = ALIGN (0x4)
                0x00000f30                __fini_array_end = .
                0x00000f30                . = ALIGN (0x4)
                0x00000f30                __text_end = .
                [0x00000f30]                PROVIDE (__text_end, __text_end)

.vfp11_veneer   0x00000f30        0x0
 .vfp11_veneer  0x00000000        0x0 linker stubs

.v4_bx          0x00000f30        0x0
 .v4_bx         0x00000000        0x0 linker stubs

.iplt           0x00000f30        0x0
 .iplt          0x00000000        0x0 out/startup.o

.rel.dyn        0x00000f30        0x0
 .rel.iplt      0x00000000        0x0 out/startup.o
                0x00000f30                . = ALIGN (0x4)
                0x00000f30                __exidx_start = .
                [0x00000f30]                PROVIDE (__exidx_start, __exidx_start)

.ARM.exidx
 *(.ARM.exidx* .gnu.linkonce.armexidx.*)
                0x00000f30                . = ALIGN (0x4)
                0x00000f30                __exidx_end = .
                [0x00000f30]                PROVIDE (__exidx_end, __exidx_end)

.data           0x10000000       0x94 load address 0x00000f30
                0x10000000                . = ALIGN (0x4)
                0x00000f30                __data_init_start = LOADADDR (.data)
                [0x00000f30]                PROVIDE (__data_init_start, __data_init_start)
                0x10000000                __data_start = .
                [0x10000000]                PROVIDE (__data_start, __data_start)
                0x10000000                . = ALIGN (0x4)
 *(.data .data.* .gnu.linkonce.d.*)
 .data.kc       0x10000000        0x1 out/cvkbdarm.o
 *fill*         0x10000001        0x3 00
 .data.scan_to_keycode
                0x10000004       0x90 out/cvkbdarm.o
                0x10000094                . = ALIGN (0x4)
                0x10000094                __data_end = .
                [0x10000094]                PROVIDE (__data_end, __data_end)

.igot.plt       0x10000094        0x0 load address 0x00000fc4
 .igot.plt      0x00000000        0x0 out/startup.o

.bss            0x10000094      0x420
                0x10000094                . = ALIGN (0x4)
                0x10000094                __bss_start = .
                [0x10000094]                PROVIDE (__bss_start, __bss_start)
                0x10000094                . = ALIGN (0x4)
 *(.bss .bss.* .gnu.linkonce.b.*)
 .bss.n_clk     0x10000094        0x1 out/cvkbdarm.o
 *fill*         0x10000095        0x1 00
 .bss.prefixes  0x10000096        0x2 out/cvkbdarm.o
 .bss.scan      0x10000098        0x1 out/cvkbdarm.o
 .bss.parity    0x10000099        0x1 out/cvkbdarm.o
 *fill*         0x1000009a        0x2 00
 .bss.scan_producer
                0x1000009c        0x4 out/cvkbdarm.o
 .bss.scan_consumer
                0x100000a0        0x4 out/cvkbdarm.o
 .bss.scans     0x100000a4      0x200 out/cvkbdarm.o
 .bss.n_errs    0x100002a4        0x1 out/cvkbdarm.o
 *fill*         0x100002a5        0x3 00
 .bss.keycode_producer
                0x100002a8        0x4 out/cvkbdarm.o
 .bss.keycode_consumer
                0x100002ac        0x4 out/cvkbdarm.o
 .bss.keycodes  0x100002b0      0x100 out/cvkbdarm.o
 .bss.modifiers
                0x100003b0        0x1 out/cvkbdarm.o
 *fill*         0x100003b1        0x3 00
 .bss.cooked    0x100003b4      0x100 out/cvkbdarm.o
                0x100004b4                . = ALIGN (0x4)
 *(COMMON)
                0x100004b4                . = ALIGN (0x4)
                0x100004b4                __bss_end = .
                [0x100004b4]                PROVIDE (__bss_end, __bss_end)

.stack          0x100004b4      0x404
                0x100004b8                . = ALIGN (0x8)
 *fill*         0x100004b4        0x4 00
                0x100004b8                __stack_start = .
                [0x100004b8]                PROVIDE (__stack_start, __stack_start)
                0x100004b8                . = ALIGN (0x8)
                0x100004b8                __main_stack_start = .
                [0x100004b8]                PROVIDE (__main_stack_start, __main_stack_start)
                0x100004b8                . = (. + __main_stack_size)
                0x100004b8                . = ALIGN (0x8)
                0x100004b8                __main_stack_end = .
                [0x100004b8]                PROVIDE (__main_stack_end, __main_stack_end)
                0x100004b8                . = ALIGN (0x8)
                0x100004b8                __process_stack_start = .
                [0x100004b8]                PROVIDE (__process_stack_start, __process_stack_start)
                0x100008b8                . = (. + __process_stack_size)
 *fill*         0x100004b8      0x400 00
                0x100008b8                . = ALIGN (0x8)
                0x100008b8                __process_stack_end = .
                [0x100008b8]                PROVIDE (__process_stack_end, __process_stack_end)
                0x100008b8                . = ALIGN (0x8)
                0x100008b8                __stack_end = .
                [0x100008b8]                PROVIDE (__stack_end, __stack_end)
                0x100008b8                . = ALIGN (0x4)
                0x100008b8                __heap_start = .
                [0x100008b8]                PROVIDE (__heap_start, __heap_start)
                0x100008b8                . = ALIGN (0x4)
                0x10001000                __heap_end = __ram_end
                [0x10001000]                PROVIDE (__heap_end, __heap_end)

.stab
 *(.stab)

.stabstr
 *(.stabstr)

.debug
 *(.debug)

.line
 *(.line)

.debug_srcinfo
 *(.debug_srcinfo)

.debug_sfnames
 *(.debug_sfnames)

.debug_aranges  0x00000000       0xb8
 *(.debug_aranges)
 .debug_aranges
                0x00000000       0x20 out/startup.o
 .debug_aranges
                0x00000020       0x20 out/vectors.o
 .debug_aranges
                0x00000040       0x78 out/cvkbdarm.o

.debug_pubnames
 *(.debug_pubnames)

.debug_info     0x00000000     0x1051
 *(.debug_info .gnu.linkonce.wi.*)
 .debug_info    0x00000000       0x48 out/startup.o
 .debug_info    0x00000048       0x92 out/vectors.o
 .debug_info    0x000000da      0xf77 out/cvkbdarm.o

.debug_abbrev   0x00000000      0x2df
 *(.debug_abbrev)
 .debug_abbrev  0x00000000       0x14 out/startup.o
 .debug_abbrev  0x00000014       0x85 out/vectors.o
 .debug_abbrev  0x00000099      0x246 out/cvkbdarm.o

.debug_line     0x00000000      0x5fc
 *(.debug_line)
 .debug_line    0x00000000       0x70 out/startup.o
 .debug_line    0x00000070       0x3e out/vectors.o
 .debug_line    0x000000ae      0x54e out/cvkbdarm.o

.debug_frame    0x00000000      0x1e0
 *(.debug_frame)
 .debug_frame   0x00000000       0x2c out/vectors.o
 .debug_frame   0x0000002c      0x194 out/cvkbdarm.o
 .debug_frame   0x000001c0       0x20 /opt/gcc-arm-none-eabi-4_7-2013q1/bin/../lib/gcc/arm-none-eabi/4.7.3/armv6-m/libgcc.a(_udivsi3.o)

.debug_str      0x00000000     0xd059
 *(.debug_str)
 .debug_str     0x00000000     0x21b3 out/vectors.o
                               0x21b8 (size before relaxing)
 .debug_str     0x000021b3     0xaea6 out/cvkbdarm.o
                               0xd0e7 (size before relaxing)

.debug_loc      0x00000000      0x2cc
 *(.debug_loc)
 .debug_loc     0x00000000       0x2c out/vectors.o
 .debug_loc     0x0000002c      0x2a0 out/cvkbdarm.o

.debug_macinfo
 *(.debug_macinfo)

.debug_weaknames
 *(.debug_weaknames)

.debug_funcnames
 *(.debug_funcnames)

.debug_typenames
 *(.debug_typenames)

.debug_varnames
 *(.debug_varnames)

.note.gnu.arm.ident
 *(.note.gnu.arm.ident)

.ARM.attributes
                0x00000000       0x2d
 *(.ARM.attributes)
 .ARM.attributes
                0x00000000       0x21 out/startup.o
 .ARM.attributes
                0x00000021       0x31 out/vectors.o
 .ARM.attributes
                0x00000052       0x31 out/cvkbdarm.o
 .ARM.attributes
                0x00000083       0x1e /opt/gcc-arm-none-eabi-4_7-2013q1/bin/../lib/gcc/arm-none-eabi/4.7.3/armv6-m/libgcc.a(_udivsi3.o)
 .ARM.attributes
                0x000000a1       0x1e /opt/gcc-arm-none-eabi-4_7-2013q1/bin/../lib/gcc/arm-none-eabi/4.7.3/armv6-m/libgcc.a(_dvmd_tls.o)

/DISCARD/
 *(.note.GNU-stack)
                0x00000f30                PROVIDE (__text_size, (__text_end - __text_start))
                0x00000000                PROVIDE (__exidx_size, (__exidx_end - __exidx_start))
                0x00000094                PROVIDE (__data_size, (__data_end - __data_start))
                0x00000420                PROVIDE (__bss_size, (__bss_end - __bss_start))
                0x00000400                PROVIDE (__stack_size, (__stack_end - __stack_start))
                0x00000748                PROVIDE (__heap_size, (__heap_end - __heap_start))
OUTPUT(out/cvkbdarm.elf elf32-littlearm)

.debug_ranges   0x00000000       0x90
 .debug_ranges  0x00000000       0x10 out/vectors.o
 .debug_ranges  0x00000010       0x80 out/cvkbdarm.o

.debug_macro    0x00000000     0x2765
 .debug_macro   0x00000000       0x11 out/vectors.o
 .debug_macro   0x00000011      0x7d2 out/vectors.o
 .debug_macro   0x000007e3      0x159 out/cvkbdarm.o
 .debug_macro   0x0000093c       0x3a out/cvkbdarm.o
 .debug_macro   0x00000976       0x10 out/cvkbdarm.o
 .debug_macro   0x00000986       0x2e out/cvkbdarm.o
 .debug_macro   0x000009b4       0xa2 out/cvkbdarm.o
 .debug_macro   0x00000a56      0x20e out/cvkbdarm.o
 .debug_macro   0x00000c64       0x1c out/cvkbdarm.o
 .debug_macro   0x00000c80       0x2e out/cvkbdarm.o
 .debug_macro   0x00000cae      0x237 out/cvkbdarm.o
 .debug_macro   0x00000ee5      0x123 out/cvkbdarm.o
 .debug_macro   0x00001008     0x15c1 out/cvkbdarm.o
 .debug_macro   0x000025c9      0x19c out/cvkbdarm.o

.comment        0x00000000       0x70
 .comment       0x00000000       0x70 out/vectors.o
                                 0x71 (size before relaxing)
 .comment       0x00000000       0x71 out/cvkbdarm.o

Cross Reference Table

Symbol                                            File
ADC_IRQHandler                                    out/vectors.o
BOD_IRQHandler                                    out/vectors.o
CAN_IRQHandler                                    out/vectors.o
HardFault_Handler                                 out/vectors.o
I2C_IRQHandler                                    out/vectors.o
PIOINT0_IRQHandler                                out/cvkbdarm.o
                                                  out/vectors.o
PIOINT1_IRQHandler                                out/vectors.o
PIOINT2_IRQHandler                                out/vectors.o
PIOINT3_IRQHandler                                out/vectors.o
PendSV_Handler                                    out/vectors.o
Reset_Handler                                     out/startup.o
                                                  out/vectors.o
SSP0_IRQHandler                                   out/vectors.o
SSP1_IRQHandler                                   out/vectors.o
SVC_Handler                                       out/vectors.o
SysTick_Handler                                   out/vectors.o
TIMER16_0_IRQHandler                              out/vectors.o
TIMER16_1_IRQHandler                              out/vectors.o
TIMER32_0_IRQHandler                              out/vectors.o
TIMER32_1_IRQHandler                              out/vectors.o
UART_IRQHandler                                   out/vectors.o
WAKEUP_PIO0_0_IRQHandler                          out/vectors.o
WAKEUP_PIO0_10_IRQHandler                         out/vectors.o
WAKEUP_PIO0_11_IRQHandler                         out/vectors.o
WAKEUP_PIO0_1_IRQHandler                          out/vectors.o
WAKEUP_PIO0_2_IRQHandler                          out/vectors.o
WAKEUP_PIO0_3_IRQHandler                          out/vectors.o
WAKEUP_PIO0_4_IRQHandler                          out/vectors.o
WAKEUP_PIO0_5_IRQHandler                          out/vectors.o
WAKEUP_PIO0_6_IRQHandler                          out/vectors.o
WAKEUP_PIO0_7_IRQHandler                          out/vectors.o
WAKEUP_PIO0_8_IRQHandler                          out/vectors.o
WAKEUP_PIO0_9_IRQHandler                          out/vectors.o
WAKEUP_PIO1_0_IRQHandler                          out/vectors.o
WDT_IRQHandler                                    out/vectors.o
__Reserved_0x08_Handler                           out/vectors.o
__Reserved_0x10_Handler                           out/vectors.o
__Reserved_0x14_Handler                           out/vectors.o
__Reserved_0x18_Handler                           out/vectors.o
__Reserved_0x1C_Handler                           out/vectors.o
__Reserved_0x20_Handler                           out/vectors.o
__Reserved_0x24_Handler                           out/vectors.o
__Reserved_0x28_Handler                           out/vectors.o
__Reserved_0x30_Handler                           out/vectors.o
__Reserved_0x34_Handler                           out/vectors.o
__Reserved_0x98_Handler                           out/vectors.o
__Reserved_0x9C_Handler                           out/vectors.o
__Reserved_0xAC_Handler                           out/vectors.o
__aeabi_idiv0                                     /opt/gcc-arm-none-eabi-4_7-2013q1/bin/../lib/gcc/arm-none-eabi/4.7.3/armv6-m/libgcc.a(_dvmd_tls.o)
                                                  /opt/gcc-arm-none-eabi-4_7-2013q1/bin/../lib/gcc/arm-none-eabi/4.7.3/armv6-m/libgcc.a(_udivsi3.o)
__aeabi_ldiv0                                     /opt/gcc-arm-none-eabi-4_7-2013q1/bin/../lib/gcc/arm-none-eabi/4.7.3/armv6-m/libgcc.a(_dvmd_tls.o)
__aeabi_uidiv                                     /opt/gcc-arm-none-eabi-4_7-2013q1/bin/../lib/gcc/arm-none-eabi/4.7.3/armv6-m/libgcc.a(_udivsi3.o)
                                                  out/cvkbdarm.o
__aeabi_uidivmod                                  /opt/gcc-arm-none-eabi-4_7-2013q1/bin/../lib/gcc/arm-none-eabi/4.7.3/armv6-m/libgcc.a(_udivsi3.o)
__bss_end                                         out/startup.o
__bss_start                                       out/startup.o
__data_end                                        out/startup.o
__data_init_start                                 out/startup.o
__data_start                                      out/startup.o
__default_low_level_init                          out/startup.o
__main_stack_end                                  out/vectors.o
__process_stack_end                               out/startup.o
__udivsi3                                         /opt/gcc-arm-none-eabi-4_7-2013q1/bin/../lib/gcc/arm-none-eabi/4.7.3/armv6-m/libgcc.a(_udivsi3.o)
low_level_init_0                                  out/startup.o
low_level_init_1                                  out/startup.o
main                                              out/cvkbdarm.o
                                                  out/startup.o
vectors                                           out/vectors.o
